:100000000C9463000C948B000C948B000C947C0873
:100010000C947C080C947C080C948B000C948B0042
:100020000C948B000C948B000C948B000C948B0024
:100030000C948B000C948B000C948B000C948B0014
:100040000C9432080C948B000C9400080C94DA0782
:100050000C948B000C948B000C948B000C948B00F4
:100060000C948B000C948B000000000024002700EF
:100070002A0000000008000201000003040700003D
:1000800000000000000000000000230026002900FE
:1000900000000000250028002B00040404040404D0
:1000A0000404020202020202030303030303010227
:1000B00004081020408001020408102001020408F6
:1000C0001020F408F10C11241FBECFEFD4E0DEBFE6
:1000D000CDBF11E0A0E0B1E0E0E5FDE102C0059098
:1000E0000D92AC32B107D9F723E0ACE2B1E001C028
:1000F0001D92AB3DB207E1F710E0C2E6D0E004C0CC
:100100002197FE010E94950EC136D107C9F70E94C2
:10011000CF090C949B0E0C940000AF92BF92CF922B
:10012000DF92EF92FF920F931F93CF93DF936C01B7
:100130007B018B01040F151FEB015E01AE18BF0898
:10014000C017D10759F06991D601ED91FC9101904A
:10015000F081E02DC6010995892B79F7C501DF9162
:10016000CF911F910F91FF90EF90DF90CF90BF90B4
:10017000AF900895FC01538D448D252F30E0842FDE
:1001800090E0821B930B541710F0CF9608950197BF
:100190000895FC01918D828D981761F0A28DAE0FAC
:1001A000BF2FB11D5D968C91928D9F5F9F73928F33
:1001B00090E008958FEF9FEF0895FC01918D828D5F
:1001C000981731F0828DE80FF11D858D90E008952C
:1001D0008FEF9FEF0895FC01918D228D892F90E084
:1001E000805C9F4F821B91098F739927089580EC43
:1001F00092E00E94EB0021E0892B09F420E0822F9D
:10020000089580E090E0892B29F00E94F700811189
:100210000C9400000895FC01A48DA80FB92FB11D06
:10022000A35ABF4F2C91848D90E001968F7399272C
:10023000848FA689B7892C93A089B1898C9183700A
:1002400080648C93938D848D981306C00288F38903
:10025000E02D80818F7D80830895EF92FF920F9330
:100260001F93CF93DF93EC0181E0888F9B8D8C8D62
:1002700098131AC0E889F989808185FF15C09FB756
:10028000F894EE89FF896083E889F9898081837019
:10029000806480839FBF81E090E0DF91CF911F91C8
:1002A0000F91FF90EF900895F62E0B8D10E00F5FE9
:1002B0001F4F0F731127E02E8C8D8E110CC00FB6BF
:1002C00007FCFACFE889F989808185FFF5CFCE0157
:1002D0000E940B01F1CFEB8DEC0FFD2FF11DE35AC6
:1002E000FF4FF0829FB7F8940B8FEA89FB898081DA
:1002F0008062CFCFCF93DF93EC01888D8823B9F054
:10030000AA89BB89E889F9898C9185FD03C0808120
:1003100086FD0DC00FB607FCF7CF8C9185FFF2CF9D
:10032000808185FFEDCFCE010E940B01E9CFDF91E7
:10033000CF91089590E0FC01EE58FF4F2491FC010D
:10034000E255FF4F3491FC01E656FF4FE491EE2356
:10035000C9F0222339F0233001F1A8F4213019F13A
:10036000223029F1F0E0EE0FFF1FE057FF4FA5917B
:10037000B4918FB7F894EC91611126C030953E236B
:100380003C938FBF08952730A9F02830C9F024305E
:1003900049F7809180008F7D03C0809180008F7726
:1003A00080938000DFCF84B58F7784BDDBCF84B5A9
:1003B0008F7DFBCF8091B0008F778093B000D2CF3C
:1003C0008091B0008F7DF9CF3E2BDACFCF93DF93B2
:1003D00090E0FC01E255FF4F249186569F4FFC01AF
:1003E00084918823D1F090E0880F991FFC01E8598F
:1003F000FF4FA591B491FC01E057FF4FC591D491F7
:1004000061110EC09FB7F8948C91E22FE0958E2376
:100410008C932881E223E8839FBFDF91CF910895D9
:100420008FB7F894EC91E22BEC938FBFF6CF2FB7F8
:10043000F89460914D0270914E0280914F0290911C
:1004400050022FBF08952091530230915402281773
:10045000390771F49091510280915202981741F03E
:10046000E0915102F0E0E85FFD4F808190E0089557
:100470008FEF9FEF08950895EF92FF920F931F93D0
:10048000CF93DF93DC015C96ED90FC905D97E114D7
:10049000F10479F481E090E013969C938E93129787
:1004A00090E080E0DF91CF911F910F91FF90EF904E
:1004B00008955196ED91FC91529750968C915097DA
:1004C000982F90950FB75E962C915E97122F127011
:1004D00021FD6095F8942081112319F1282B2083A8
:1004E000E7012197F1F728E0462F50E0308160FFC7
:1004F0001AC0382B3083E7012197F1F7BA017595BF
:100500006795215089F7112381F0808189238083A9
:100510000FBF5C968D919C910197F1F781E090E07F
:10052000C1CF2923DCCF3923E5CF9081892BEFCFB1
:1005300020915302309154022817390761F48091B9
:1005400052022091510290E0805C9F4F821B9109E2
:100550008F739927089590E080E0089520915302C9
:100560003091540228173907B9F4909151028091C3
:100570005202981789F0E0915102F0E0E85FFD4FD8
:1005800080812091510230E02F5F3F4F2F7333273E
:100590002093510290E008958FEF9FEF089590E02F
:1005A00080E00895FC01369620E08FEF9FEF26173C
:1005B00091F03191832738E0AC0141705527969531
:1005C0008795452B21F041E0842740EA942731505C
:1005D00099F72F5FECCF9827892798270895CF9216
:1005E000DF92FF920F931F93CF93DF9300D000D041
:1005F000CDB7DEB78C016C0186E4C80ED11CD601E4
:10060000FC906F2DC8010E94D202F801EF0DF11D80
:100610009683E1E0EF0DE00FF12FF11D8683F39457
:10062000F394F601F082D80113968C91823018F081
:1006300061E00E949A01F80180819181D6014C917C
:1006400050E0DC01ED91FC910280F381E02DB801D6
:100650006A5F7F4F0995F8018381823058F180816C
:100660009181DC01ED91FC910680F781E02D0995E7
:10067000F801E65AFF4F80819181A281B38189837D
:100680009A83AB83BC8389819A81AB81BC81AC01A5
:10069000BD01415051096109710949835A836B8336
:1006A0007C83892B8A2B8B2B71F760E0F801838187
:1006B0000E949A01D8018D919C91DC01ED91FC91F1
:1006C0000284F385E02D099597FFF4CFF60110829F
:1006D0000E941702F801EA5AFF4F608371838283F8
:1006E00093833A97808191810196918380830F90C3
:1006F0000F900F900F90DF91CF911F910F91FF906E
:10070000DF90CF900895FF920F931F93CF93DF93C5
:10071000EC018B81823018F060E00E949A018E011A
:100720000A5B1F4FD8011C92F12C88819981DC0152
:10073000ED91FC910084F185E02D0995892BB9F0AC
:1007400088819981DC01ED91FC910284F385E02D93
:100750000995F8019081FE01E90FF11D86839F5FE5
:10076000D8019C93903408F3FF24F394DECFFE016C
:10077000E65BFF4F80819181019691838083FF200A
:1007800071F0C25BDF4F88819981019699838883DC
:100790008DEFDF91CF911F910F91FF900895F80198
:1007A0008081F7CF4F925F926F927F928F929F924C
:1007B000AF92BF92CF92DF92EF92FF920F931F936F
:1007C000CF93DF93EB018A018093570290935802F5
:1007D00070935C0260935B0224E020935602309198
:1007E00055024091590250915A02609161037091F3
:1007F0005F03711123C0611121C06FEF630F673F69
:1008000008F0E2C0D093A603C093A503309363031E
:10081000209364039093650380936603509367036A
:100820004093680386E08093A3038DE593E00E94E4
:10083000EF0281E0809361031092620358E0C52EBD
:1008400051E0D52EBB24BA9480916103882309F42A
:10085000BBC080915D0390915E03DC01ED91FC9142
:100860000084F185E02D0995982E0E941702409092
:10087000B3035090B4036090B5037090B603AB011E
:10088000BC0144195509660977098091AD0390911F
:10089000AE03B0E0A0E084179507A607B70770F491
:1008A00010926103B09262038091AB039091AC030C
:1008B00001969093AC038093AB03C6CF992021F2AD
:1008C0008091A403981669F09092A4030E941702E5
:1008D0006093AF037093B0038093B1039093B2031E
:1008E000B3CF0E9417024090AF035090B0036090C6
:1008F000B1037090B20364197509860997096530D0
:1009000071058105910508F49FCF1092A4038DE530
:1009100093E00E94830386301CF410926103C4CFDD
:100920006091A303862E912C62508DE593E00E9486
:10093000D202F401E35AFC4F248135812327322768
:1009400023272817390761F08091AB039091AC03FE
:1009500001969093AC038093AB031092610374CF24
:100960008091640387FDF0CFE0E0F1E09191891779
:1009700009F4B3C2CE16DF06C9F7E6CF80E0909146
:100980006503891750F7282F269530E0220F331F73
:10099000E091A503F091A603E20FF31F908141813E
:1009A000A82FB0E0A35ABC4F19962C9130E080FFDD
:1009B00007C0892E922E9401318320838F5FDFCF71
:1009C000E12C2E29342BF8CF6881798190E080E0EA
:1009D000CB0177276627CA80DB80F12CE12C6C29BC
:1009E0007D298E299F29D8016D937D938D939C93AA
:1009F000139720E030E04AE754E40E94280E0E945A
:100A00007F0D7B836A83998388838CEB91E090933D
:100A1000AA028093A90286E28093BF0280916102BC
:100A200090916202DC01ED91FC910084F185E02D52
:100A30000995882381F09091A8028917E9F08093A5
:100A4000A8020E9417026093B3027093B4028093CD
:100A5000B5029093B602DF91CF911F910F91FF9055
:100A6000EF90DF90CF90BF90AF909F908F907F904E
:100A70006F905F904F9008950E9417020091B3020B
:100A80001091B4022091B5023091B602601B710B37
:100A9000820B930B6530710581059105E0F2109290
:100AA000A80281E692E00E94830380936602873069
:100AB00094F290916702809163029813CCCF609179
:100AC000A702C62FD0E0625081E692E00E94D202D7
:100AD000CF59DD4F2C813D8123273227232728172B
:100AE000390769F08091AF029091B002019690931E
:100AF000B0028093AF02CFEFC0936602ACCF2091DB
:100B00006802E0E0F1E088E091E03191321709F409
:100B10000CC28E179F07C9F78091AF029091B00267
:100B200001969093B0028093AF02C1E020582093C9
:100B30006802C093690283E08093A70281E692E095
:100B40000E94EF02D9CF8091690290916A029827A2
:100B500089279827AC01F4E056954795FA95E1F777
:100B600080916B0290916C02982789279827A4E0C6
:100B700096958795AA95E1F7840F951F0CC08091F3
:100B8000690290916A02982789279827E4E0969550
:100B90008795EA95E1F79091BF029817C0F4C2E0FB
:100BA000C5CF8091690290916A0298278927F3CF77
:100BB0008091690290916A0298278927982740912D
:100BC0006B0250916C02542745275427D5CF0E94C1
:100BD00017026093B7027093B8028093B9029093A2
:100BE000BA0210926602E0916802E150E03108F02A
:100BF00032CFF0E0E250FA4F0C94950E0E060E063E
:100C000089068906BD06ED062B052B052B052B0550
:100C10002B052B052B052B05FC064C078091690243
:100C200090916A0298278927982700916B0210916A
:100C30006C02102701271027980173E0369527953D
:100C40007A95E1F7E22FE801C770DD27209711F0D0
:100C5000E1E0E20FE093690223E02093A702F0E0D5
:100C6000EF59FD4F1086080F191F30E0C12CD12C11
:100C70007601C3940817190791F1E22FF0E0B7014C
:100C8000A601032E04C0440F551F661F771F0A9448
:100C9000D2F7EF59FD4FB680DC0153E0B695A7952A
:100CA0005A95E1F7AE7FB170A454BE4F6D907C9021
:100CB000B82FBF709B2ED30102C0B695A7959A940A
:100CC000E2F7A0FF09C04B2946833F5F383010F0A0
:100CD0002F5F30E00196CECF40954B21F5CFCD2B45
:100CE000B1F42093A70281E692E0DF91CF911F91AA
:100CF0000F91FF90EF90DF90CF90BF90AF909F90BB
:100D00008F907F906F905F904F900C94EF022F5FC9
:100D1000E8CF8091690290916A0298278927982FDD
:100D200020916B0230916C0232272327322F330F30
:100D300030936902E3E0280F3327331F82E08E0FE0
:100D4000A92FB0E0A217B307ACF4AA0FBB1FA4549D
:100D5000BE4F4C9111965C91AE2FB0E0AF59BD4F94
:100D600016965C93EF5FF0E0EF59FD4F46839F5F6F
:100D7000E82FE4CFE093A702B6CF2091690230912B
:100D80006A02322723273227F90173E0F695E795A7
:100D90007A95E1F7EE7FF170E454FE4F4081518186
:100DA0002F7081E090E0A0E0B0E004C0880F991FB0
:100DB000AA1FBB1F2A95D2F720916B022F3F41F447
:100DC000842B952B9183808386E08093A7028BCF21
:100DD0008095909584239523F5CFE0916A02F0E009
:100DE000EE0FFF1FE454FE4F80916B0290916C0256
:100DF000982789279827E6CF8091690290916A0207
:100E000098278927982720916B0230916C0232270E
:100E100023273227280F391F10E007E0C12CD12CDF
:100E20007601C3942817390779F2FC0143E0F6955F
:100E3000E7954A95E1F7EE7FF170E454FE4F482FB5
:100E40004F704601570104C0880C991CAA1CBB1C9A
:100E50004A95D2F7A401C081D181A02FB0E0AF594B
:100E6000BD4F1696AC91B0E0012E02C0B595A79586
:100E70000A94E2F7A0FF0BC04C2B5D2B51834083FB
:100E80001F5F183010F00F5F10E00196CBCF409538
:100E900050954C235D23F2CFE0916A0240916C02A1
:100EA00010926B0286E08093A702A1E6B2E0F0E028
:100EB000EE0FFF1FE454FE4F80E01296481709F42E
:100EC00012CF1B962C911B971C969C911C97322F2E
:100ED000292F219331938F5FF0CF813008F43DCDDE
:100EE000833008F44BCD853008F037CD90E080E0BA
:100EF00023E0309165033695831708F02ECDE22F5D
:100F0000F0E0AC01440F551FA091A503B091A603DA
:100F1000A40FB51FE35AFC4F46813781542F432F4E
:100F20004D935C932E5F0196E4CFEFEFE20FE0313B
:100F300008F04DCEF0E0E156F84F0C94950EA30565
:100F4000A305D805D805BF05D105E705E705E705E1
:100F5000E705E705E705E705E705A305D805CF930E
:100F6000DF93EC018B81823038F061E00E94E60172
:100F700060E08B810E949A0188819981DC01ED916A
:100F8000FC910284F385E02D099597FFF5CFFE01D2
:100F9000EA5BFF4F108231961082379611821082E1
:100FA000329711821082C65BDF4F19821882DF915F
:100FB000CF9108951F920F920FB60F9211242F9385
:100FC0003F934F935F936F937F938F939F93AF93D1
:100FD000BF93EF93FF9380EC92E00E940B01FF918F
:100FE000EF91BF91AF919F918F917F916F915F91A1
:100FF0004F913F912F910F900FBE0F901F9018951A
:101000001F920F920FB60F9211242F938F939F93DD
:10101000EF93FF93E091D002F091D1028081E091B3
:10102000D602F091D70282FD1BC090818091D90237
:101030008F5F8F732091DA02821741F0E091D9021D
:10104000F0E0E054FD4F958F8093D902FF91EF912E
:101050009F918F912F910F900FBE0F901F90189519
:101060008081F4CF1F920F920FB60F9211242F930D
:101070003F938F939F93AF93BF9380914D02909135
:101080004E02A0914F02B091500230914C0223E0E9
:10109000230F2D3758F50196A11DB11D20934C0249
:1010A00080934D0290934E02A0934F02B093500252
:1010B0008091480290914902A0914A02B0914B025E
:1010C0000196A11DB11D8093480290934902A093FF
:1010D0004A02B0934B02BF91AF919F918F913F9184
:1010E0002F910F900FBE0F901F90189526E8230F99
:1010F0000296A11DB11DD2CF1F920F920FB60F9273
:1011000011242F933F934F935F936F937F938F930C
:101110009F93AF93BF93EF93FF93E0915302F091AE
:101120005402309749F0A685B7858585968D91FF45
:1011300014C09C918923A1F4FF91EF91BF91AF91CD
:101140009F918F917F916F915F914F913F912F91DF
:101150000F900FBE0F901F9018959C91892361F7F7
:10116000A389B4899C918589809589238C938689EC
:1011700097890197F1F7608D718DA685B7855585A3
:1011800038E020E0CB010197F1F7822F90E09595B0
:101190008795282F4C91452309F02068315091F70D
:1011A000868D81FD20958091520290E001968F738B
:1011B000992730915102381799F0A0915202B0E06E
:1011C000A85FBD4F2C9380935202828D938D01971F
:1011D000F1F7A389B4898C919589892B8C93ACCF35
:1011E000868D8160868FF1CF1092C3021092C20269
:1011F00088EE93E0A0E0B0E08093C4029093C50233
:10120000A093C602B093C7022CE031E03093C10234
:101210002093C00225EC30E03093CD022093CC0225
:1012200024EC30E03093CF022093CE0220EC30E06B
:101230003093D1022093D00221EC30E03093D302DE
:101240002093D20222EC30E03093D5022093D402D6
:1012500026EC30E03093D7022093D6021092D902C8
:101260001092DA021092DB021092DC021092BF039D
:101270001092BE038093C0039093C103A093C20356
:10128000B093C3038EE191E09093BD038093BC03C0
:101290001092D3031092D2031092D5031092D4036C
:1012A0001092D7031092D6031092D9031092D8034C
:1012B0006091DA036E7F6D7F6093DA0366956170EB
:1012C00081E0682785E00E949A0161E085E00E9444
:1012D000E601E3EBF0E0E491E093CC03EFE9F0E02A
:1012E000E491F0E0EE0FFF1FE057FF4F85919491DE
:1012F0009093CE038093CD0360E086E00E94E601E8
:101300008091DA0381FD04C061E086E00E949A01C9
:1013100086E08093C803E4EBF0E0E491E093C90336
:10132000E0EAF0E0E491F0E0EE0FFF1FEA57FF4F34
:10133000859194919093CB038093CA0380EC92E0C3
:1013400090935E0380935D0310925F0322E02093ED
:10135000600388EE93E09093AE038093AD03109208
:10136000B7031092B8031092B9031092BA034CEB72
:1013700053E050936202409361022093630227E09E
:10138000209364029093B2028093B1021092BB0248
:101390001092BC021092BD021092BE020895789481
:1013A00084B5826084BD84B5816084BD85B582606A
:1013B00085BD85B5816085BD80916E00816080931B
:1013C0006E00109281008091810082608093810084
:1013D0008091810081608093810080918000816094
:1013E000809380008091B10084608093B1008091EF
:1013F000B00081608093B00080917A008460809317
:101400007A0080917A00826080937A0080917A00DD
:10141000816080937A0080917A00806880937A005E
:101420001092C100109284011092850110928601E1
:101430001092870110928C0110928D0110928E01F2
:1014400010928F0110929C0110929D0110929E01AA
:1014500010929F011092A4011092A5011092A60172
:101460001092A7011092AC011092AD011092AE0142
:101470001092AF0110925D0210925E0210925F0214
:101480001092600261E08DE00E94E6011092D703A5
:101490001092D6031092D5031092D4031092D30366
:1014A0001092D2038DEC90E09093D9038093D803EF
:1014B0009091C803963108F047C025E530E030939D
:1014C000D3032093D2032BEC30E03093D503209349
:1014D000D40320E930E03093D7032093D603209142
:1014E000680084E0983048F031E09E3008F430E045
:1014F00081E001C0880F3A95EAF7822B809368005B
:101500002DE630E0983050F02BE630E09E3030F0A1
:101510002CE630E0963110F030E020E03093D0033C
:101520002093CF03292F30E0983008F030C281E0BB
:1015300001C0880F9A95EAF78093D1038091D80370
:101540009091D9030197F1F78091D6039091D70339
:10155000892B49F1E0915302F091540283E0EC3B76
:10156000F80709F1309739F0A389B4899C918589EE
:10157000809589238C938091DA038E7F8093DA03A0
:1015800010925202109251028CEB93E0909354020D
:1015900080935302E091CF03F091D003808190912A
:1015A000D103892B8083E091D002F091D10282E0B7
:1015B0008083E091CC02F091CD021082E091CE02C6
:1015C000F091CF028FEC80831092D802E091D40288
:1015D000F091D50286E08083E091D202F091D302AF
:1015E000808180618083E091D202F091D30280817A
:1015F00088608083E091D202F091D302808180687C
:101600008083E091D202F091D30280818F7D80832C
:101610008DE593E00E94AF0781E692E00E94AF075C
:101620008AEF90E09093AE038093AD0381E08093C6
:10163000550282E090E090935A02809359021092F2
:101640000302109202021092010210920002C0E006
:10165000D0E04CE251E06CEB71E090E080E00E9461
:10166000D20344E351E060EC71E082E090E00E943C
:10167000D2034CE351E064EC71E084E090E00E941E
:10168000D20344E451E068EC71E086E090E00E940F
:10169000D203C0904401D0904501E0904601F09003
:1016A000470120919C0130919D0140919E015091F4
:1016B0009F01C701B6010E94230E1816D4F4C092F0
:1016C0009C01D0929D01E0929E01F0929F0120E04A
:1016D00030E04AE754E4C701B6010E94280E0E9498
:1016E0007F0D7093F7016093F6019093F50180935D
:1016F000F4014CE451E06CEC71E088E090E00E9471
:10170000D203C0904C01D0904D01E0904E01F0907A
:101710004F012091A4013091A5014091A601509163
:10172000A701C701B6010E94230E1816D4F4C09277
:10173000A401D092A501E092A601F092A70120E0B9
:1017400030E04AE754E4C701B6010E94280E0E9427
:101750007F0D7093FB016093FA019093F9018093E0
:10176000F80144E551E060ED71E08AE090E00E940C
:10177000D203C0905401D0905501E0905601F090F2
:1017800057012091AC013091AD014091AE015091D3
:10179000AF01C701B6010E94230E1816D4F4C092FF
:1017A000AC01D092AD01E092AE01F092AF0120E029
:1017B00030E04AE754E4C701B6010E94280E0E94B7
:1017C0007F0D7093FF016093FE019093FD01809364
:1017D000FC014CE551E064ED71E084E390E00E948F
:1017E000D203C0905C01D0905D01E0905E01F0906A
:1017F0005F01A7019601609184017091850180913C
:101800008601909187010E947A0D87FF1AC0C092CD
:101810008401D0928501E0928601F092870120E058
:1018200030E04AE754E4C701B6010E94280E0E9446
:101830007F0D7093EB016093EA019093E90180932F
:10184000E80144E651E068ED71E08CE390E00E942D
:10185000D2034CE651E06CED71E084E090E00E9430
:10186000D20344E751E060EE71E08EE390E00E9425
:10187000D2034CE751E064EE71E086E591E00E940E
:10188000D203C0905D02D0905E02E0905F02F090C3
:10189000600220E030E0A901C701B6010E947A0D84
:1018A000811182C01092EF011092EE011092ED01B1
:1018B0001092EC0180917C0190917D01A0917E01BC
:1018C000B0917F0180935D0290935E02A0935F02CE
:1018D000B093600244E951E060EF71E086E490E08B
:1018E0000E94D203609100027091010290E080E0BA
:1018F000CB0177276627009102021091030230E0A6
:1019000020E0602B712B822B932B20E030E0A9018B
:101910000E947A0D882381F1109203021092020234
:10192000109201021092000210928401109285011F
:10193000109286011092870110928C0110928D01F5
:1019400010928E0110928F0110929C0110929D01B5
:1019500010929E0110929F011092A4011092A50175
:101960001092A6011092A7011092AC011092AD0145
:101970001092AE011092AF01209709F46ACE0E9436
:10198000F700882309F465CE0E94000062CE9E30E5
:1019900040F42850310981E001C0880F2A95EAF708
:1019A000CBCD2E503109F7CFA701960160917C0174
:1019B00070917D0180917E0190917F010E940D0DBB
:1019C00020E030E04AE754E40E94280E0E947F0D98
:1019D0007093EF016093EE019093ED018093EC0121
:1019E00079CF8EE191E09093BD038093BC03809109
:1019F0005302909154028C5B934071F4E091CF03B9
:101A0000F091D00390818091D103809589238083C8
:101A1000109254021092530208955058BB27AA27DF
:101A20000E94250D0C94E90D0E94DB0D38F00E94F8
:101A3000E20D20F039F49F3F19F426F40C94D80DF0
:101A40000EF4E095E7FB0C94D20DE92F0E94FA0DFD
:101A500058F3BA17620773078407950720F079F4E3
:101A6000A6F50C941C0E0EF4E0950B2EBA2FA02DAB
:101A70000B01B90190010C01CA01A0011124FF273B
:101A8000591B99F0593F50F4503E68F11A16F04036
:101A9000A22F232F342F4427585FF3CF4695379535
:101AA0002795A795F0405395C9F77EF41F16BA0BFA
:101AB000620B730B840BBAF09150A1F0FF0FBB1FA8
:101AC000661F771F881FC2F70EC0BA0F621F731FF1
:101AD000841F48F4879577956795B795F7959E3F4E
:101AE00008F0B0CF9395880F08F09927EE0F9795DF
:101AF000879508950E94AE0D08F481E008950E9434
:101B0000020E88F09F5798F0B92F9927B751B0F07F
:101B1000E1F0660F771F881F991F1AF0BA95C9F771
:101B200014C0B13091F00E941C0EB1E008950C94E5
:101B30001C0E672F782F8827B85F39F0B93FCCF398
:101B4000869577956795B395D9F73EF490958095EE
:101B5000709561957F4F8F4F9F4F0895990F0008A3
:101B6000550FAA0BE0E8FEEF16161706E807F9076F
:101B7000C0F012161306E407F50798F0621B730B0A
:101B8000840B950B39F40A2661F0232B242B252B8B
:101B900021F408950A2609F4A140A6958FEF811D2E
:101BA000811D089597F99F6780E870E060E00895CF
:101BB0009FEF80EC089500240A9416161706180665
:101BC0000906089500240A94121613061406050641
:101BD0000895092E0394000C11F4882352F0BB0FD2
:101BE00040F4BF2B11F460FF04C06F5F7F4F8F4F35
:101BF0009F4F089557FD9058440F551F59F05F3F70
:101C000071F04795880F97FB991F61F09F3F79F01E
:101C100087950895121613061406551FF2CF4695A0
:101C2000F1DF08C0161617061806991FF1CF869522
:101C30007105610508940895E894BB276627772706
:101C4000CB0197F908950E94AE0D08F48FEF089527
:101C50000E943B0E0C94E90D0E94DB0D38F00E94AF
:101C6000E20D20F0952311F00C94D20D0C94D80DB8
:101C700011240C941D0E0E94FA0D70F3959FC1F370
:101C8000950F50E0551F629FF001729FBB27F00D2A
:101C9000B11D639FAA27F00DB11DAA1F649F66277F
:101CA000B00DA11D661F829F2227B00DA11D621FCE
:101CB000739FB00DA11D621F839FA00D611D221F88
:101CC000749F3327A00D611D231F849F600D211D6C
:101CD000822F762F6A2F11249F5750409AF0F1F0EF
:101CE00088234AF0EE0FFF1FBB1F661F771F881F58
:101CF00091505040A9F79E3F510580F00C94D20DB1
:101D00000C941D0E5F3FE4F3983ED4F386957795CF
:101D10006795B795F795E7959F5FC1F7FE2B880FFD
:101D2000911D9695879597F90895EE0FFF1F0590E1
:101D3000F491E02D099410E0C2E6D0E004C0FE0169
:101D40000E94950E2196C336D107C9F7F894FFCFAC
:101D50000102030405060F10000000002D018D0094
:101D6000BA007A01EB00C900DD00000000003C026F
:0C1D70008D00CF023B029802AE0223025D
:00000001FF
